:040000002EEF12F0DD
:1000080000C016F001C015F0E1CF1BF0E2CF1CF0E4
:10001800F5CF1AF0F8CF17F0F7CF18F0F6CF19F0A0
:100028009DA29CD19EA29AD19E92010E4024006E60
:10003800000E4120016E00C040F001C041F0800E6A
:10004800006E800E4118005C02E14050050802E293
:10005800406A416A010E00016115016E0150000AF3
:10006800D8A4A9D00A0E605DD8B0A5D07DD0899A51
:100078000F0E010123155E6E720E5E24F66E3D0EA4
:10008800F76E000EF722000EF86E000EF822090037
:10009800F5CF00F0425000108A6E89808BD089908D
:1000A80023C100F00032009E0032009E0032009E04
:1000B8000032009E00C05EF0720E5E24F66E3D0EA9
:1000C800F76E000EF722000EF86E000EF8220900F7
:1000D800F5CF00F0425000108A6E89826BD0899269
:1000E800390E42108A6E898465D089944250630F14
:1000F8008A6E89865FD0010189960F0E24155E6E7F
:10010800720E5E24F66E3D0EF76E000EF722000E9C
:10011800F86E000EF8220900F5CF00F042500010EA
:100128008A6E898847D0899824C100F00032009EE1
:100138000032009E0032009E0032009E00C05EF039
:10014800720E5E24F66E3D0EF76E000EF722000E5C
:10015800F86E000EF8220900F5CF00F042500010AA
:100168008A6E898A27D026D0000E411802E1000E37
:100178004018D8B47CD7000E411802E1010E40188F
:100188008EE0000E411802E1020E4018A8E0000EB1
:10019800411802E1030E4018A8E0000E411802E1E0
:1001A800040E4018A8E0000E411802E1050E4018A0
:1001B800BAE0D9D7D2D0A9D00101899A0F0E30154B
:1001C8005E6E720E5E24F66E3D0EF76E000EF7221E
:1001D800000EF86E000EF8220900F5CF00F042502C
:1001E80000108A6E8980B9D0899030C100F0003241
:1001F800009E0032009E0032009E0032009E00C029
:100208005EF0720E5E24F66E3D0EF76E000EF7225B
:10021800000EF86E000EF8220900F5CF00F04250EB
:1002280000108A6E898299D0010189920F0E2A15D1
:100238005E6E720E5E24F66E3D0EF76E000EF722AD
:10024800000EF86E000EF8220900F5CF00F04250BB
:1002580000108A6E898481D089942AC100F0003206
:10026800009E0032009E0032009E0032009E00C0B8
:100278005EF0720E5E24F66E3D0EF76E000EF722EB
:10028800000EF86E000EF8220900F5CF00F042507B
:1002980000108A6E898661D0010189960F0E2B1590
:1002A8005E6E720E5E24F66E3D0EF76E000EF7223D
:1002B800000EF86E000EF8220900F5CF00F042504B
:1002C80000108A6E898849D089982BC100F00032C5
:1002D800009E0032009E0032009E0032009E00C048
:1002E8005EF0720E5E24F66E3D0EF76E000EF7227B
:1002F800000EF86E000EF8220900F5CF00F042500B
:1003080000108A6E898A29D028D0000E411802E18F
:10031800000E4018D8B450D7000E411802E1010E63
:100328004018D8B461D7000E411802E1020E4018F7
:10033800D8B47AD7000E411802E1030E40188CE0B9
:10034800000E411802E1040E4018A6E0000E411804
:1003580002E1050E4018B8E0D7D79E929EAA6AD04F
:100368009DAA68D057EC0DF000C0DBF1ABA20ED00F
:10037800AB98010E0101D525006E000ED621016E45
:1003880000C0D5F101C0D6F1AB88DB6BABA411D0AE
:100398000101AB9E010ED525006E000ED621016E1F
:1003A80000C0D5F101C0D6F1AB8E57EC0DF000C0FE
:1003B800DBF10101DB510D0A07E0BC51000802E145
:1003C800BB517F0801E31ED0010EB96F000EBA6F52
:1003D800350EB525E16E010EB621E26EE66A9D9AEC
:1003E800B5C1BBF1B6C1BCF1B56BB66BBC51000869
:1003F80002E1BB517F0804E2020EB96F000EBA6F2A
:100408009D9218D0B96BBA6B350EB525E16E010E09
:10041800B621E26EDBC1E6FFB5C1BBF1B6C1BCF1E6
:10042800010EB525006E000EB621016E00C0B5F1B3
:1004380001C0B6F11AC0F5FF17C0F8FF18C0F7FFE2
:1004480019C0F6FF16C000F015C001F01BC0E1FF8F
:060458001CC0E2FF1100D0
:10045E000B820BAE39EF02F0036802680168006888
:08046E000A360232FF0E1200F3
:080476000AAE029E000E120006
:10047E000B840BAE4AEF02F0010E036E026A016AA4
:0A048E00006A0A360232FF0E120067
:0E049800ACB202D00000FCD72AC2ADFF1200A9
:0C04A60072B201D0FDD72AC273FF120011
:0E04B200026A016A006A086A036A000E1200FC
:1004C000F250026EF29E0500FF6A0150FE6E00506F
:0804D000FD6E02BEF28E120067
:1004D800C7B409D01F0EC514016E0150000A03E10C
:0A04E800010E006E01D0006A120040
:1004F2000CB0BBEF02F00CA261EF03F00E6A000E2B
:100502000264D2EF02F0F00E0214D8A49DEF02F0C2
:10051200023A01380F0B02260138F00B016E003847
:100522000F0B01260038F00B006E08380F0B002667
:100532000838F00B086E0E84D89002BEB6EF02F0B7
:1005420008360036013602360E2A02BEB6EF02F037
:1005520008360036013602360E2A02BEB6EF02F027
:1005620008360036013602360E2A0E50036457EF63
:1005720003F0035E0BBC08AE5CEF03F0D880800E84
:1005820008640030000E002201220222D8A05CEF93
:1005920003F0023201320032034A61EF03F05CEFF2
:1005A20003F001C002F000C001F008C000F0086AC8
:1005B200000E0E86026409EF03F0F00E0214D8A4B6
:1005C200F1EF02F0023A01380F0B02260138F00B6C
:1005D200016E00380F0B01260038F00B006E0E84FE
:1005E200D89002BEB6EF02F00036013602360E2A6D
:1005F20002BEB6EF02F00036013602360E2A02BE05
:10060200B6EF02F00036013602360E2AB6EF02F0DD
:1006120001C002F000C001F0006A000E0E960E88C2
:10062200026436EF03F0F00E0214D8A421EF03F0B7
:10063200023A01380F0B02260138F00B016E0E84CC
:10064200D89002BEB6EF02F0013602360E2A02BE82
:10065200B6EF02F0013602360E2A02BEB6EF02F003
:10066200013602360E2AB6EF02F001C002F0016A2C
:10067200000E0E86026466EF03F0F00E0214D8A498
:1006820045EF03F0023A0E84D89002BEB6EF02F0B4
:1006920002360E2A02BEB6EF02F002360E2A02BE61
:1006A200B6EF02F002360E2AB6EF02F0010E0C6E21
:1006B200E5DE69EF03F0020E0C6EDCDE69EF03F09B
:1006C200040E0C6ECBDE69EF03F0080E0C6EF0DE4A
:0206D200120014
:0806D4000B6A0B86FF0E1200F9
:1006DC00086A096A100E0C6E01340836093604508B
:1006EC00085E0550D8A0053C095ED8B007D0045070
:1006FC0008260550D8B0053C0926D890003601369E
:06070C000C2EEAD71200DA
:100712000B6A0A6A096A00500402F4CF09F0F3CFA7
:1007220008F001500502F4CF0BF0F3CF0AF00050AD
:100732000502F3500926F4500A22E86A0B220150FE
:100742000402F3500926F4500A22E86A0B2208C078
:1007520000F009C001F00AC002F00BC003F0120061
:100762000C6A0E6A0250D8A4CAEF03F001C002F06C
:1007720000C001F0006A0E860250D8A4CAEF03F04E
:1007820001C002F0016A0E960E880250D8B4DCEF66
:1007920003F00E50035ED8A4D8A0E1EF03F0D89086
:1007A20002BEE6EF03F0003601360236032ED1EF29
:1007B20003F0E1EF03F0010E0C6E7ADEE9EF03F0D5
:1007C200020E0C6E5BDEE9EF03F0040E0C6E52DEDD
:0207D200120013
:1007D4000B800BAEF6EF03F0026A0AAEFF0E026E58
:0C07E400016E006E0A360232FF0E120099
:1007F00002012451390806E3300E245D03E3010EA3
:08080000006E01D0006A120035
:10080800025006180E6E086A096A0B6A03500764DC
:10081800F7EF04F006500A6E068E028E03500B6E38
:100828000750036E000E0B6447EF04F00B50075E91
:10083800D8B4E8EF04F0070E0764B6EF04F0075EDB
:1008480000C008F001C000F002C001F0026A074EC3
:10085800E8EF04F007648BEF04F0075E00C008F0CF
:1008680001C000F0016A074EE8EF04F0076469EF81
:1008780004F0075E00C008F0006A074EE8EF04F0D5
:10088800076450EF04F00AC002F005C001F004C08C
:1008980000F0086A11EF06F0030E07645BEF04F03E
:1008A800075E08380F0B086E074EE8EF04F0D89083
:1008B8000832074EE8EF04F0D8900832074EE8EF08
:1008C80004F0D8900832E8EF04F0030E07647AEFDA
:1008D80004F0075E08380F0B086E0038F00B082686
:1008E80000380F0B006E074EE8EF04F0D890003286
:1008F8000832074EE8EF04F0D89000320832074E6D
:10090800E8EF04F0D89000320832E8EF04F0030E64
:100918000764A2EF04F0075E08380F0B086E003872
:10092800F00B082600380F0B006E0138F00B00267C
:1009380001380F0B016E074EE8EF04F0D890013232
:1009480000320832074EE8EF04F0D8900132003246
:100958000832074EE8EF04F0D8900132003208322E
:10096800E8EF04F0030E0764D3EF04F0075E0838DD
:100978000F0B086E0038F00B082600380F0B006EBE
:100988000138F00B002601380F0B016E0238F00B0E
:10099800012602380F0B026E074EE8EF04F0D890DC
:1009A8000232013200320832074EE8EF04F0D890E4
:1009B8000232013200320832074EE8EF04F0D890D4
:1009C8000232013200320832096A000E0EAEDCEF44
:1009D80005F0081E001E011E021E082A0022012220
:1009E8000222DCEF05F00750D8A4FDEF04F011EF68
:1009F80006F0096A02C00AF0028E068E0750035CF0
:100A0800076ED8B4CFEF05F0070E07649DEF05F029
:100A1800075E0450096E0550046E0650056E066A9E
:100A2800074ECFEF05F0070E076472EF05F0075E7B
:100A38000450096E0550046E056A074ECFEF05F0A5
:100A4800070E076450EF05F0075E0450096E046A4C
:100A5800074ECFEF05F0070E076437EF05F00AC021
:100A680002F011EF06F0030E076442EF05F0075E8F
:100A780009380F0B096E074ECFEF05F0D8900932F1
:100A8800074ECFEF05F0D8900932074ECFEF05F0AB
:100A9800D8900932CFEF05F0030E076461EF05F037
:100AA800075E09380F0B096E0438F00B0926043865
:100AB8000F0B046E074ECFEF05F0D89004320932C1
:100AC800074ECFEF05F0D89004320932074ECFEF2A
:100AD80005F0D89004320932CFEF05F0030E076411
:100AE80089EF05F0075E09380F0B096E0438F00B23
:100AF800092604380F0B046E0538F00B0426053858
:100B08000F0B056E074ECFEF05F0D8900532043273
:100B18000932074ECFEF05F0D8900532043209327A
:100B2800074ECFEF05F0D890053204320932CFEFE7
:100B380005F0030E0764BAEF05F0075E09380F0BDE
:100B4800096E0438F00B092604380F0B046E0538BB
:100B5800F00B042605380F0B056E0638F00B05263A
:100B680006380F0B066E074ECFEF05F0D890063209
:100B7800053204320932074ECFEF05F0D89006321D
:100B8800053204320932074ECFEF05F0D89006320D
:100B9800053204320932086A000E0EAEDCEF05F0A9
:100BA800091E041E051E061E092A04220522062205
:100BB800095008260450002205500122065002223E
:100BC8000EBEF3EF05F0D8A002EF06F002320132B4
:100BD80000320832033E02EF06F00CEF06F0D8B000
:100BE80007EF06F0000E081E001E011E021E082A4E
:100BF8000022012202220A7E07EF06F0010E0C6E87
:100C080074DC13EF06F0020E0C6E6FDC13EF06F0C7
:100C1800040E0C6E20DC13EF06F0000E0C6E1200B2
:100C28005AC024F25BC025F25CC026F25DC027F2F0
:100C3800C582C5A21FD05A505B105C105D1019E028
:100C4800020124512511261127110CE1D9C1E1FF18
:100C5800DAC1E2FF060EE66ED7C100F0D8C101F096
:100C68002BDC08D0010E0201245F000E255B265BF9
:060C7800275BDFD712002C
:100C7E005AC026F25BC027F25CC028F25DC029F292
:100C8E009E96C5869EB620D05A505B105C105D10A5
:100C9E001AE0020126512711281129110DE1D9C19F
:100CAE00E1FFDAC1E2FF030EE66ED7C100F0D8C154
:100CBE0001F060EC02F008D0010E0201265F000E7A
:100CCE00275B285B295BDED70201C9CF25F22451B1
:100CDE00000A02E1C58A01D0C59A9E96C5885AC0FF
:100CEE0026F25BC027F25CC028F25DC029F29EB6E8
:100CFE0020D05A505B105C105D101AE00201265194
:100D0E002711281129110DE1D9C1E1FFDAC1E2FF46
:100D1E00030EE66ED7C100F0D8C101F060EC02F010
:100D2E0008D0010E0201265F000E275B285B295BAF
:080D3E00DED725C200F012000F
:040D4600C58412004E
:100D4A00086A080E0C6E003408360450085ED8B0E3
:0E0D5A0002D00826D89000360C2EF5D71200D5
:100D68005AC026F25BC027F25CC028F25DC029F2A7
:100D78000201246B256B2551120802E124518E08CB
:100D880009E36CEC02F0005201E004D00201244BAC
:100D9800252BF1D70201120E255D02E18F0E245D8D
:100DA80003E37B0E006E25D0C580C5A021D05A5024
:100DB8005B105C105D101BE02651271128112911CA
:100DC8000FE1D9C1E1FFDAC1E2FF050EE66ED7C136
:100DD80000F0D8C101F060EC02F0010E006E09D0FD
:100DE800010E0201265F000E275B285B295BDDD719
:040DF800006A12007B
:100DFC009E9624C2C9FF5AC025F25BC026F25CC085
:100E0C0027F25DC028F2C7A422D05A505B105C10A8
:100E1C005D101CE0020125512611271128110FE14C
:100E2C00D9C1E1FFDAC1E2FF040EE66ED7C100F0D2
:100E3C00D8C101F060EC02F0010E006E3BD0010E47
:100E4C000201255F000E265B275B285BDCD75AC0AE
:100E5C0025F25BC026F25CC027F25DC028F29EB67C
:100E6C0022D05A505B105C105D101CE00201255121
:100E7C002611271128110FE1D9C1E1FFDAC1E2FFD8
:100E8C00040EE66ED7C100F0D8C101F060EC02F0A0
:100E9C00010E006E0FD0010E0201255F000E265BC5
:100EAC00275B285BDCD7C5BC02D0006A03D0C584A5
:060EBC00020E006E1200A0
:100EC20000C008F00150006E016A026A036A0B6AF0
:100ED2000C6A016A026A036A960E036E0A6A00AE1F
:100EE20079EF07F0081E001E082AD8B4002A0A8EDD
:100EF20000C001F008C000F0086A026A31DC12008A
:100F020002011D6B1C5109081BE20A0E046E1CC271
:100F120000F01ADF00C01DF200C01DF21D371D9146
:100F22001D371D911D371D911D371D910A0E046E2F
:100F32001CC200F009DF08C000F000501D1302D0EF
:0A0F42001CC21DF21DC200F01200D7
:100F4C000DDFD00E0201246F53DF1CC224F250DFE0
:100F5C0065DED10E0201246F4BDF0201246B89DEAA
:0C0F6C0000C01DF2EADE1DC200F0120001
:060F7800067E46DC1200BB
:100F7E000D0E02012A6F4CEC02F00A0E02012A6FCE
:060F8E004CEC02F0120021
:100F94001CC2E9FF1DC2EAFFEECF1EF2000E0201E1
:100FA4001F6F000E1F6F000E1F1902E1200E1E1985
:100FB40007E0000E1F1902E1090E1E1901E003D01B
:100FC4001C4B1D2BE5D7206B216B226B236B000E72
:100FD4001F1902E12D0E1E1905E1224B232B1C4B78
:100FE4001D2B08D0000E1F1902E12B0E1E1902E161
:100FF4001C4B1D2B1CC2E9FF1DC2EAFFEECF1EF2E3
:10100400000E1F6F000E1F6F1EC224F2F8EC03F0D7
:10101400005219E020C200F021C201F00A0E046E51
:10102400000E056E89EC03F0300E1E5D026E000E9C
:101034001F59036E02500024206F03500120216FBA
:101044001C4B1D2BD7D72251231108E02051000837
:10105400006E21C201F0000E015604D020C200F03F
:0610640021C201F01200A0
:0C106A003A0E0D6E0D2EFED70000120095
:1010760002011F6B030E1F5D0AE21F511D25E16E63
:10108600000E1E21E26E200EE66E1F2BF3D71F51B7
:101096001D25E16E000E1E21E26EE66A1F071F5136
:1010A6001D25206F000E1E21216F0A0E046E1CC224
:1010B60000F048DE08C000F0300E002620C2E1FF36
:1010C60021C2E2FF00C0E6FF0A0E046E1CC200F059
:1010D60039DE00C01CF20050000A01E102D01F07F1
:0410E600DED712003F
:1010EA003EDED00E0201246F84DE1CC224F281DEB1
:0A10FA001DC224F27EDE22DE120089
:101104000201206B050E205D0AE220511E25E16ECE
:10111400000E1F21E26E200EE66E202BF3D7205125
:101124001E25E16E000E1F21E26EE66A20072051A3
:101134001E25216F000E1F21226F0A0E046E000E61
:10114400056E1CC200F01DC201F06EEC03F008C075
:1011540000F009C001F0300E002621C2E1FF22C2D6
:10116400E2FF00C0E6FF0A0E046E000E056E1CC20C
:1011740000F01DC201F06EEC03F000C01CF201C0CF
:101184001DF2000E011802E1000E001801E102D068
:061194002007CDD7120078
:10119A001CC2F6FF1DC2F7FF1EC2F8FF0900F5CFF9
:1011AA0000F0005212E01CC2F6FF1DC2F7FF1EC279
:1011BA00F8FF0900F5CF2AF24CEC02F0010E020109
:0C11CA001C27000E1D231E23E3D712007B
:1011D60002011F6B1CC2E9FF1DC2EAFFEECF1EF221
:1011E6001E51000A0FE01EC22AF24CEC02F0020168
:1011F6001F2B1F511C25E96E000E1D21EA6EEECF36
:061206001EF2EED71200FB
:10120C001CC200F00032009E0032009E0032009E94
:10121C000032009E1DC2E1FF1EC2E2FF300E002410
:10122C00E66E010E02011D25E16E000E1E21E26E1E
:10123C000F0E1C15006E300E002600C0E6FF020ECD
:0E124C001D25E16E000E1E21E26EE66A120004
:10125A000A6A0350D8A40A800750D8A40A820A50FE
:10126A00D8B490EF09F0030AD8B449EF09F00AB0EC
:10127A0044EF09F006AE8EEF09F08CEF09F002AEEA
:10128A008CEF09F08EEF09F00250800B0A6E029E75
:10129A000650800B069E0A18D8B45AEF09F00A5075
:1012AA00D8B48CEF09F08EEF09F00750035CD8B47C
:1012BA0064EF09F0D8A080EF09F086EF09F0065034
:1012CA00025CD8B46EEF09F0D8A080EF09F086EF7F
:1012DA0009F00550015CD8B478EF09F0D8A080EF86
:1012EA0009F086EF09F00450005CD8B490EF09F0D9
:1012FA00D8B086EF09F00A52D8B48EEF09F08CEF15
:10130A0009F00A52D8B48CEF09F08EEF09F0D880B0
:0E131A001200D8901200D880D8841200120061
:101328000450000A12E10550000A0FE10650000AB5
:101338000CE10750000A09E1FF0E006EFF0E016E76
:101348007F0E026EFF0E036EA8D0086A096A075066
:10135800D8B43FEF0AF00350D8B444EF0AF0025073
:1013680006180A6E028E068E0E6A02C008F001C0C8
:101378000CF000C00DF004500D5E0550D8A0053CDF
:101388000C5E0650D8A0063C085E086A0C6A0D6A16
:10139800D8A0D6EF09F0D8900232013200320832D4
:1013A800010E0E6E0750035ED8A0E3EF09F07E0E23
:1013B8000E240326D8B049EF0AF0E9EF09F07E0EB3
:1013C8000E240326D8A04EEF0AF0180E0B6E0D3629
:1013D8000C3608360036013602360E360450005EEA
:1013E8000550D8A0053C015E0650D8A0063C025E18
:1013F80006340E120EA004EF0AF00D800FEF0AF06B
:10140800045000260550D8B0053C01260650D8B037
:10141800062802260D900B2EEBEF09F035EF0AF0A7
:10142800D8900036013602360E360450005E05505C
:10143800D8A0053C015E0650D8A0063C025E0634E2
:101448000E10010B0D26D8B00C2AD8B4082AD8A43F
:1014580035EF0AF008320C320D32032AD8B449EFBE
:101468000AF00AAE089E0850026E0C50016E0D502C
:10147800006E51EF0AF0010E6AEC03F051EF0AF02A
:10148800020E59EC02F051EF0AF0040E2FEC02F0B4
:0C14980051EF0AF0080E3FEC02F01200C9
:1014A400A69C1DC2AAFF1CC2A9FFA69EA680A8CF07
:0414B40000F0120032
:1014B8000B6A0350D8B4A2EF0AF002500A6E028EEB
:1014C8008E0E035E03AEA6EF0AF0036C080E035CF3
:1014D800D8A081EF0AF0036E013602C001F0026A5B
:1014E800080E035CD8A081EF0AF0036E0136016A8A
:1014F8000350D8A4D8908BEF0AF00350D8B48BEFE0
:101508000AF0D89002320132032E85EF0AF00BBCA4
:1015180001A098EF0AF0D8A098EF0AF0012AD8B4F1
:10152800022A02BEB5EF0AF00AAEBBEF0AF0021EAD
:10153800011E012AD8B4022ABBEF0AF0026A016A26
:10154800BBEF0AF00B800BAEBFEF0AF0026A0AAEDF
:10155800BFEF0AF0FF0E026E016E0A360232BFEFCD
:101568000AF0010E0C6EEAEC03F0C1EF0AF0000E6F
:101578000C6EC1EF0AF0FF0E0C6E0150006E0250A7
:04158800016E1200DE
:10158C00086A096A000E076203644BEF0BF0025005
:10159C0006180A6E075003267E0ED8A0DCEF0AF060
:1015AC00035ED8B050EF0BF0E0EF0AF0035ED8A06A
:1015BC0055EF0BF0028E068E02C00EF001C00BF040
:1015CC0000C00DF000500402F4CF0CF001500502E5
:1015DC00F4CF00F0F3CF08F00402F3500C26F450D3
:1015EC000822000E00220D500502F3500C26F45078
:1015FC000822000E002202500402F3500826F45078
:10160C00002202500502016A000E0122F35000264E
:10161C00F45001220D500602F3500826F45000221B
:10162C00026A000E012202220B500602F350002621
:10163C00F4500122000E02220E500602F350012635
:10164C00F450022202BE33EF0BF00836003601369E
:10165C0002360306D8B455EF0BF046EF0BF0D880EA
:10166C00800E08640030000E002201220222D8A055
:10167C0046EF0BF0023201320032034A50EF0BF00E
:10168C000AAE029E000E58EF0BF0010E59EC02F060
:10169C0058EF0BF0020E2FEC02F058EF0BF0040E8B
:0616AC003FEC02F0120009
:1016B200B4EC06F0D00E0201246FFEEC06F002013B
:1016C200246BFEEC06F014EC06F0D10E0201246F3E
:1016D200FEEC06F0010E0201246F3FEC06F000C0A2
:1016E20030F1010E0201246F3FEC06F000C02AF136
:1016F200010E0201246F3FEC06F000C02BF1010E37
:101702000201246F3FEC06F000C069F000500608A9
:1017120002E20001696B010E0201246F3FEC06F048
:1017220000C0FAF0010E0201246F3FEC06F000C087
:10173200F9F00201246B3FEC06F000C0FDF0A3ECCF
:1017420006F02BC11CF2430E02011D6F000E1E6F2C
:101752005CDD3A0E456E2AC11CF2460E1D6F000E6C
:101762001E6F53DD3A0E486E30C11CF2490E1D6FDA
:10177200000E1E6F4ADD4B6AFAC01CF24C0E1D6F42
:10178200000E1E6F42DD2D0E4E6EF9C01CF24F0E82
:101792001D6F000E1E6F39DD2D0E516EFDC01CF245
:1017A200520E1D6F000E1E6F30DD546A0101F7519B
:1017B200010A1AE14C0E02011C6F000E1D6F0ADDB8
:1017C200D60E1C6F3D0E1D6F000E1E6FE5DC430E24
:1017D20002011C6F000E1D6FFDDCD60E1C6F3D0E4C
:0A17E2001D6F000E1E6FD8DC120010
:1017EC000101FC6BFD6BF7C1FEF1000EF7BFFF0EA4
:1017FC00FF6F800EF719006E800E000A005C0AE283
:10180C00FC4BFD2BF7510008FE6FFF6B000EF7BF72
:10181C00FF0EFF5BFEC11CF2F8C11DF2F9C11EF2F6
:10182C0024DC040E0101FA6F000EFB6F000E006E3B
:10183C00FB51005C02E1FA51000819E2FA51F8255B
:10184C00E16EFB51F921E26E010EFA5D006E000EA5
:10185C00FB59016E0050F825E96E0150F921EA6E32
:10186C00EECFE6FF010EFA5F000EFB5BDFD7F8C18F
:10187C00E1FFF9C1E2FF200EE66EFC51FD111AE00A
:10188C00FA6BFB6BFA51F825E96EFB51F921EA6E04
:10189C00EE50200A03E1FA4BFB2BF4D7010EFA5F52
:1018AC00000EFB5BFA51F825E16EFB51F921E26E5B
:0618BC002D0EE66E120085
:1018C200D80E0101E46F040EE56F000EE66F000E04
:1018D200E76F680EE86F0D0EE96F000EEA6F000EFB
:1018E200EB6F280EE06F0C0EE16F000EE26F000E40
:1018F200E36F7E0EBD6F0C0EBE6F240EBF6F020E25
:10190200C06FFC0ECD6F0D0ECE6F240ECF6F020E88
:10191200D06F460EC96F0D0ECA6F000ECB6F000E50
:10192200CC6F949894968B988B9694889486C79E45
:08193200C79C380EC66E1200BE
:10193A000101FD6BFE6BF7C101F2F8C102F2800EE4
:10194A00F819006E800E005C02E1000EF75D0CE2F1
:10195A00010EFD6F000EFE6FF75100080201016FC4
:10196A00F8C102F2000E025701C21CF202C21DF2B5
:10197A00F9C11EF2FAC11FF282EC08F0060E01014B
:10198A00FB6F000EFC6F000E006EFC51005C02E162
:10199A00FB51000819E2FB51F925E16EFC51FA21CD
:1019AA00E26E010EFB5D006E000EFC59016E0050E6
:1019BA00F925E96E0150FA21EA6EEECFE6FF010E33
:1019CA00FB5F000EFC5BDFD7F9C1E1FFFAC1E2FF62
:1019DA00200EE66EFD51FE111AE0FB6BFC6BFB510B
:1019EA00F925E96EFC51FA21EA6EEE50200A03E16C
:1019FA00FB4BFC2BF4D7010EFB5F000EFC5BFB518B
:101A0A00F925E16EFC51FA21E26E2D0EE66E120006
:101A1A00980E0101C56F040EC66F2A0EC76F020E1B
:101A2A00C86FAE0EC16F1A0EC26F000EC36F000EE2
:101A3A00C46FFF0ED16FFF0ED26F000ED36F000E70
:101A4A00D46FFF0EDC6FFF0EDD6F000EDE6F000E2F
:101A5A00DF6FAC8A900EAB6E948E949C9EAA03D0D4
:081A6A00AECF00F0FBD7120023
:101A7200806A0F01386B800E926E929C899C396B42
:101A8200816A936AF18EFF0E616E8A9E8A8E426A25
:101A9200796A786A826A3A6B3A85870E946E948084
:0C1AA2009492606A428F429B42891200BD
:101AAE00AECF01F0ABA202D0AB98AB8801C000F074
:021ABE00120014
:101AC0000900F5CFE6FF0006FBE10106F9E112008F
:101AD0000101FD51000805E3070EFE6F000EFF6FC8
:101AE00015D0FD51160806E2170E0201016F000E17
:101AF000026F08D00101FD51010F0201016F026B5D
:101B0000000E022301C2FEF102C2FFF10201FEC17A
:101B100009F2FFC10AF2036B046B046A056A066AE4
:101B2000076AF7C100F0F8C101F0F9C102F0FAC18B
:101B300003F02DEC09F0010ED8B0000E006E00523B
:101B40000AE0FBC1E1FFFCC1E2FF2D0EE66E0101E0
:101B5000FB4BFC2BF97FF7C104F0F8C105F0F9C18C
:101B600006F0FAC107F0006A016A026A036A2DEC06
:101B700009F0010ED8B0000E006E005237E0000EE2
:101B8000046E000E056E000E066E7F0E076EF7C126
:101B900000F0F8C101F0F9C102F0FAC103F02DEC38
:101BA00009F0010ED8B0000E006E00521FE0F7C120
:101BB00000F0F8C101F0F9C102F0FAC103F0000E23
:101BC000046E000E056E200E066E820E076EDEDCC1
:101BD00000C0F7F101C0F8F102C0F9F103C0FAF159
:101BE000010E0201035F000E045BC9D7000E046EF4
:101BF000000E056E200E066E820E076EF7C100F015
:101C0000F8C101F0F9C102F0FAC103F02DEC09F0BE
:101C1000000ED8B0010E006E00521EE0000E046EE1
:101C2000000E056E200E066E820E076EF7C100F0E4
:101C3000F8C101F0F9C102F0FAC103F094EC09F027
:101C400000C0F7F101C0F8F102C0F9F103C0FAF1E8
:101C50000201034B042BCAD7020103510927045187
:101C60000A23010E056F000E066F000E0B6F000EAB
:101C70000C6F000E0D6F7F0E0E6F800E0619006E3A
:101C8000800E0A19005C02E10951055D1EE2000E9A
:101C9000046E000E056E200E066E820E076E0BC2DD
:101CA00000F00CC201F00DC202F00EC203F094EC81
:101CB00009F000C00BF201C00CF202C00DF203C02B
:101CC0000EF20201054B062BD8D7000E046E000E53
:101CD000056E000E066E800E076E0BC200F00CC281
:101CE00001F00DC202F00EC203F094EC09F0F7C14E
:101CF00004F0F8C105F0F9C106F0FAC107F004ECF0
:101D000004F000C0F7F101C0F8F102C0F9F103C01E
:101D1000FAF1000E046E000E056E200E066E820EA5
:101D2000076E2DEC09F0000ED8B0010E006E0052C7
:101D30000CE0000E0101F76F000EF86F000EF96F56
:101D40007F0EFA6F0201034B042B0201800E04196F
:101D5000006E800E005C02E1000E035D3CE2FBC100
:101D6000E1FFFCC1E2FF300EE66E0101FB4BFC2BF4
:101D7000FBC1E1FFFCC1E2FF2E0EE66EFB4BFC2B2C
:101D8000800E02010A19006E800E005C02E1000E56
:101D9000095D04E20951035F0A51045BFF0E056F00
:101DA000FF0E066F800E0419006E800E0619005C8F
:101DB00002E10551035D0FE2FBC1E1FFFCC1E2FF5F
:101DC000300EE66E0101FB4BFC2B010E0201055F9C
:101DD000000E065BE7D7056B066B800E0619006EDA
:101DE000800E0A19005C02E10951055D67E2F7C146
:101DF00000F0F8C101F0F9C102F0FAC103F05CECA7
:101E00000AF000C007F201C008F2300E0026FBC144
:101E1000E1FFFCC1E2FF00C0E6FF0101FB4BFC2B30
:101E200002010651041902E10351051909E1FBC140
:101E3000E1FFFCC1E2FF2E0EE66E0101FB4BFC2B25
:101E400007C200F008C201F061EC07F000C00BF21D
:101E500001C00CF202C00DF203C00EF200C004F08B
:101E600001C005F002C006F003C007F0F7C100F0A2
:101E7000F8C101F0F9C102F0FAC103F0BCEC07F0BF
:101E800000C0F7F101C0F8F102C0F9F103C0FAF1A6
:101E9000000E046E000E056E200E066E820E076E9A
:101EA000C6EC0AF000C0F7F101C0F8F102C0F9F188
:101EB00003C0FAF10201054B062B8FD7FBC1E1FFEE
:081EC000FCC1E2FFE66A12001A
:101EC800A6A202D00000FCD7A69CF8C1AAFFF7C1C1
:101ED800A9FFF9C1A8FFA69EA684F2CF00F0F29E42
:101EE800550EA76EAA0EA76EA68200BE02D0F29E5D
:101EF80001D0F28EA694A1B802D00000FCD7A19818
:021F08001200C5
:101F0A00F7C119F2000E02011A6F19C21CF21AC2A5
:101F1A001DF252EC0AF000C01BF20050000A01E167
:101F2A0029D0800E006E800E1A19005C02E1195148
:101F3A00FE0801E21FD00101F7510201195D006E8E
:101F4A00000E1A59016EF80E0024E16E010E0120EE
:101F5A00E26E1BC2E6FF340E0C6EF10E0D6E0D2EF4
:101F6A00FED70C2EFCD700000000194B1A2B1B5170
:101F7A00000ACBE1F80E1925E16E010E1A21E26E74
:0C1F8A00E66AF80E006E010E016E1200F7
:101F9600020E0101F76F000EF86FFB6BFC6B9D9A4A
:101FA600350EBB25E16E010EBC21E26EE66A000E1F
:101FB600BC5D02E1150EBB5DD8B0E6D0000E006E2A
:101FC600BC51005C02E1BB511208D8B0DDD0670EEF
:101FD60002011C6F3D0E1D6F000E1E6FCDEC08F04A
:101FE600BBC11CF2BCC11DF26C0E02011E6F000EBD
:101FF6001F6F82EC08F06C0E1C6F000E1D6FEBEC71
:1020060008F0BFEC07F0020E0101F96F000EFA6F3F
:10201600BC51FA5D02E1BB51F95D33E2350EF9259B
:10202600E96E010EFA21EA6EEE503B0A27E1350E03
:10203600F925E16E010EFA21E26EE66A8C0EFB25A9
:10204600FD6F000EFC21FE6F350EF72502011C6F99
:10205600010E0101F82102011D6FCAEC07F0FDC156
:10206600E1FFFEC1E2FF00C0E6FF010E0101F92516
:10207600F76F000EFA21F86FFB4BFC2BF94BFA2B8E
:10208600C7D78C0EFB25FD6F000EFC21FE6F350EAB
:10209600F72502011C6F010E0101F82102011D6FD7
:1020A600CAEC07F0FDC1E1FFFEC1E2FF00C0E6FF9A
:1020B6008CC0FAF08DC0F9F08EC0FDF08FC069F0CB
:1020C60000018F5106080AE2696B870E02011C6F38
:1020D6003B0E1D6F000E1E6FCDEC08F090C02BF16D
:1020E60091C02AF102011C6B1D6B75EC08F02AC128
:1020F6001CF281EC07F000C01DF2010E1C6F75EC9E
:1021060008F02BC11CF281EC07F000C01DF2020E94
:102116001C6F75EC08F069C01CF281EC07F000C07A
:102126001DF2030E1C6F75EC08F0FAC01CF281EC70
:1021360007F000C01DF2040E1C6F75EC08F0F9C024
:102146001CF281EC07F000C01DF2050E1C6F75EC49
:1021560008F0FDC01CF281EC07F000C01DF2060E6F
:102166001C6F75EC08F0070E02011C6F100E1D6F38
:1021760075EC08F00B0E02011C6F3C0E1D6F000E75
:102186001E6FCDEC08F012D02E0E02011C6F3A0E17
:102196001D6F000E1E6FCDEC08F0640E02011C6F61
:0E21A6003B0E1D6F000E1E6FCDEC08F01200F8
:1021B400F7C102F0F8C103F002C000F003C001F05F
:1021C400024A032A00C0E9FF01C0EAFFEE5201E01F
:1021D400F3D70101F751025C006EF8510358016E08
:0A21E400010E005E000E015A120009
:1021EE0002011C6BA6EC07F000C030F1010E0201DB
:1021FE001C6FA6EC07F000C02AF1020E02011C6F44
:10220E00A6EC07F000C02BF1030E02011C6FA6EC2A
:10221E0007F000C069F00050060802E20001696B89
:10222E00040E02011C6FA6EC07F000C0FAF0050EBA
:10223E0002011C6FA6EC07F000C0F9F0060E0201B9
:0C224E001C6FA6EC07F000C0FDF01200B1
:10225A000101FB6B050EFB5D0AE2FB51F925E16EFC
:10226A00000EFA21E26E300EE66EFB2BF3D7FB511D
:10227A00F925E16E000EFA21E26EE66AFB07000E0E
:10228A00F81902E1000EF7192CE0FB51F925FC6F51
:10229A00000EFA21FD6F0A0E046E000E056EF7C1DC
:1022AA0000F0F8C101F06EEC03F008C000F009C0BC
:1022BA0001F0300E0026FCC1E1FFFDC1E2FF00C0C3
:1022CA00E6FFFB070A0E046E000E056EF7C100F06A
:1022DA00F8C101F06EEC03F000C0F7F101C0F8F1AB
:0422EA00CED7120039
:1022EE003E0EBA6E9D82FA0EBB6EC00EF26E1200DC
:1022FE000101B56BB66B000EB65D02E17F0EB55DEA
:10230E0012E2350EB525E16E010EB621E26EE66AD9
:10231E00010EB525006E000EB621016E00C0B5F19E
:10232E0001C0B6F1E8D7356BB56BB66BB76BB86B52
:10233E00BB6BBC6BB96BBA6BAECFDBF1DB6B9D8A43
:02234E0012007B
:10235000CC0E0101316F230E326FF70E336F010E79
:10236000346FC26A5F50F715006E0AE05F50F715D0
:102370000F01426F428F42BD02D00000FCD702D055
:102380000F01426B591C006E0050C11659500101DB
:10239000F715006E0050C1120F0EC012C08EC28021
:0223A000120029
:1023A2000050086E0150006E016A026A036A0B6AED
:1023B2000C6A960E036E0A6A00C001F008C000F0B3
:0A23C200086A026AB1EC03F0120091
:1023CC00830EC216F7C100F0003600900036009064
:1023DC000050C21235EC08F0C282C2A201D0FDD767
:1023EC00C4CF01F0006A00C0F8F101C0F9F1C3508C
:1023FC000012000E011200C0F8F101C0F9F1000E3C
:10240C000014026E0150800B036E000E031802E1E3
:10241C00000E021803E00101F86BF96BF8C100F033
:06242C00F9C101F01200ED
:10243200F7C100F00032009E0032009E0032009E82
:102442000032009E0A0E0002F3CF01F00F0E0101CE
:0A245200F715006E0150002612007D
:10245C00F4EC1EF0D38CD38AD398D392D3909B6A8E
:10246C009B8C39EC0DF08B82426A00016A6B6B6BB2
:10247C00000E6B5D02E17F0E6A5D0AE2350E6A2585
:10248C00E16E010E6B21E26EE66A6A4B6B2BF0D7A4
:10249C006A6B6B6B000E6B5D02E11F0E6A5D0AE2EC
:1024AC006C0E6A25E16E000E6B21E26EE66A6A4BD9
:1024BC006B2BF0D76A6B6B6B000E6B5D02E1630EDE
:1024CC006A5D0AE2950E6A25E16E000E6B21E26EE2
:1024DC00E66A6A4B6B2BF0D7950EFB6F000EFC6F08
:1024EC00B886B06A440EAF6EAC840DEC0DF0050EE0
:1024FC000B6E0F0E0C6EF10E0D6E0D2EFED70C2EFC
:10250C00FCD70B2EFAD70C0E02012A6F4CEC02F002
:10251C00150E0B6E4B0E0C6EBE0E0D6E0D2EFED7E9
:10252C000C2EFCD70B2EFAD70000BFEC07F0060ED2
:10253C0002011C6F3D0E1D6F000E1E6FCDEC08F0DE
:10254C0000016A6B6B6B000E6B5D02E10A0E6A5D3B
:10255C001CE2030E006E000E016E6AC004F06BC02C
:10256C0005F089EC03F01D0E0024E96E000E01202D
:10257C00EA6EEECF1CF2EECF1DF2EECF1EF2CDECDA
:10258C0008F000016A4B6B2BDED7290E0B6E960EF2
:10259C000C6E7F0E0D6E0D2EFED70C2EFCD70B2E57
:1025AC00FAD7BFEC07F0950E0001FB6F000EFC6F25
:1025BC00626B636B606B616B646B656B686B406AC1
:1025CC00416A899C2A0E02011C6F3C0E1D6F000E85
:1025DC001E6FCDEC08F0600E0101F76F90DC00C0AF
:1025EC0066F001C067F00D0E0024E16E000E0120B4
:1025FC00E26EE66A0B0E0001662502011C6F000EEE
:10260C000001672102011D6FCAEC07F000C03EF00B
:10261C0001C03FF000C01CF201C01DF26C0E1E6F19
:10262C00000E1F6F82EC08F06C0E1C6F000E1D6FFD
:10263C00EBEC08F0BFEC07F0140E02011C6F3B0E24
:10264C001D6F000E1E6FCDEC08F0700E0101F76FC0
:10265C0056DC00C066F001C067F00D0E0024E16E80
:10266C00000E0120E26EE66A0B0E000166250201E7
:10267C001C6F000E0001672102011D6FCAEC07F0F0
:10268C0000C055F001C056F000C01CF201C01DF294
:10269C006C0E1E6F000E1F6F82EC08F06C0E1C6F20
:1026AC00000E1D6FEBEC08F0100E00016625E16EBC
:1026BC00000E6721E26EE66A0E0E662502011C6FA3
:1026CC00000E0001672102011D6FCAEC07F000C06B
:1026DC0057F001C058F000C01CF201C01DF26C0E86
:1026EC001E6F000E1F6F82EC08F06C0E1C6F000E3C
:1026FC001D6FEBEC08F0BFEC07F0500E02011C6FE5
:10270C00360E1D6F000E1E6FCDEC08F0900E010101
:10271C00F76F85EC0FF000C066F001C067F0040E97
:10272C0000241C6F000E01201D6FCAEC07F000C0C6
:10273C0026F100C0F7F1000E00BEFF0E0101F86F8C
:10274C006C0EF96F000EFA6F9DEC0CF06C0E020122
:10275C001C6F000E1D6FEBEC08F0BFEC07F0F10ED8
:10276C0002011C6F3C0E1D6F000E1E6FCDEC08F0AD
:10277C00140EC86E61EC0CF0460E02011C6F3C0E80
:10278C001D6F000E1E6FCDEC08F00E0E02011C6FBB
:10279C00400E1D6F75EC08F082B042D0DC0E0201C9
:1027AC001C6F3C0E1D6F000E1E6FCDEC08F002016D
:1027BC001C6B500E1D6F75EC08F0010E02011C6FA6
:1027CC00590E1D6F75EC08F00E0E02011C6F81EC9A
:1027DC0007F000C01DF2020E1C6F75EC08F0030E22
:1027EC0002011C6F020E1D6F75EC08F0040E020145
:1027FC001C6F010E1D6F75EC08F0050E02011C6FAD
:10280C00050E1D6F75EC08F0120E02011C6F81ECA9
:10281C0007F000C01DF2060E1C6F75EC08F009D015
:10282C002B0E02011C6F3D0E1D6F000E1E6FCDECAA
:10283C0008F0010E0101F76F59EC0BF0BFEC07F03B
:10284C00C30E02011C6F390E1D6F000E1E6FCDECF6
:10285C0008F0180E0101F76F75DD510E02011C6FA7
:10286C00390E1D6F000E1E6FCDEC08F0BFEC07F09B
:10287C00406A416A010127933C0E02011C6F3D0E18
:10288C001D6F000E1E6FCDEC08F08B92290E0B6E97
:10289C00960E0C6E7F0E0D6E0D2EFED70C2EFCD7E9
:1028AC000B2EFAD78B82010E0101F76F59EC0BF04E
:1028BC00BFEC07F0190E02011C6F3D0E1D6F000ED0
:1028CC001E6FCDEC08F055C01CF256C01DF26C0EFC
:1028DC0002011E6F000E1F6F82EC08F06C0E1C6F55
:1028EC00000E1D6FEBEC08F0200E0101EC6F650E75
:1028FC00ED6F740EEE6F200EEF6F4D0EF06F610EDC
:10290C00F16F780EF26F200EF36F480EF46F3D0EE0
:10291C00F56FF66BEC0E02011C6F010E1D6FEBECEC
:10292C0008F057C01CF258C01DF26C0E1E6F000E42
:10293C001F6F82EC08F06C0E1C6F000E1D6FEBEC21
:10294C0008F0BFEC07F00101286B296B0001646BE8
:10295C00656B01012C6B2D6B2E6B2F6BCADCC1DCF4
:10296C00F28C0001626B636BF28E0101279FBFEC4E
:10297C0007F00101F76B59EC0BF030C1F7F153DDA7
:10298C0000C060F02AC1F7F14EDD00C061F02BC130
:10299C00F7F149DD00C068F0000160513A080AE225
:1029AC00010127B307D0000160510101251902E193
:1029BC0027838B92000160510101251908E0898C55
:1029CC0060C025F127A302D027938B8201D0899C6C
:1029DC000E0EF76FF5DC010126510026000E26BF06
:1029EC00FF0E012200C01CF101C01DF100500001BE
:1029FC006427015065230101284B292B800E006EA2
:102A0C00800E2919005C02E128510708D8B034D196
:102A1C00DC0E02011C6F3D0E1D6F000E1E6FCDEC07
:102A2C0008F04C0E02011C6F000E1D6FEBEC08F051
:102A3C00D90E1C6F3D0E1D6F000E1E6FCDEC08F0F5
:102A4C00430E02011C6F000E1D6FEBEC08F0DF0E45
:102A5C001C6F3D0E1D6F000E1E6FCDEC08F0000EAE
:102A6C00006E5850005C03E157500001685D1FE296
:102A7C00000E565C03E100016851555C18E2000140
:102A8C006151000A14E1000E006E3F50005C02E13F
:102A9C003E50605D0CE2800E426ED20E02011C6F45
:102AAC003D0E1D6F000E1E6FCDEC08F00AD0426A71
:102ABC00CE0E02011C6F3D0E1D6F000E1E6FCDEC75
:102ACC0008F03B0E02012A6F4CEC02F064C000F0DF
:102ADC0065C001F060DCCD0E046ECC0E056E4C0EA4
:102AEC00066E780E076EC6EC0AF000C02CF101C021
:102AFC002DF102C02EF103C02FF164C000F065C0AF
:102B0C0001F001320032019E01320032019E01328D
:102B1C000032019E00C064F001C065F000C0F7F106
:102B2C0001C0F8F16C0E0101F96F000EFA6F2DEC7B
:102B3C0011F0E50E02011C6F3D0E1D6F000E1E6F95
:102B4C00CDEC08F06C0E02011C6F000E1D6FEBEC4F
:102B5C0008F0E20E1C6F3D0E1D6F000E1E6FCDECCB
:102B6C0008F02CC1F7F12DC1F8F12EC1F9F12FC1EC
:102B7C00FAF1FE0E0101FB6F000EFC6F020EFD6FF1
:102B8C0068EC0DF0FE0E1C6F000E1D6FEBEC08F0E8
:102B9C00CA0E1C6F3D0E1D6F000E1E6FCDEC08F0A3
:102BAC00BFEC07F0FE0E0101F76F000EF86FDAECC8
:102BBC0010F000C01EF101C01FF1020E005C026E8D
:102BCC00000E0158036EFE0E0224E96E000E032067
:102BDC00EA6EEECF02F0300E025C036E03C004F01E
:102BEC0004360490043604900436049004360490A1
:102BFC00010E005C026E000E0158036EFE0E0224E4
:102C0C00E96E000E0320EA6EEECF02F0300E025E8B
:102C1C0002500424236F050E005C026E000E015856
:102C2C00036EFE0E0224E96E000E0320EA6EEECF58
:102C3C0002F0300E025C046E04C002F00236029008
:102C4C00023602900236029002360290040E005EAA
:102C5C00000E015AFE0E0024E96E000E0120EA6EF1
:102C6C00EECF00F0300E005E00500224246F286B73
:102C7C00296B0001646B656B7FEC11F0110E0B6E10
:102C8C003C0E0C6ECB0E0D6E0D2EFED70C2EFCD703
:102C9C000B2EFAD7000EBA1902E1010EB919D8A4FD
:102CAC0016EF1BF0350EB76F010EB86FB7C1E9FF09
:102CBC00B8C1EAFFEE50480A44E1030EB725E96EAD
:102CCC00000EB821EA6EEE50700A3BE1B00E020124
:102CDC001C6F3C0E1D6F000E1E6FCDEC08F03D0EF0
:102CEC0002011C6F3B0E1D6F000E1E6FCDEC08F029
:102CFC00EB0E02011C6F3B0E1D6F000E1E6FCDEC18
:102D0C0008F0F90E02011C6F390E1D6F000E1E6FBC
:102D1C00CDEC08F05B0E02011C6F370E1D6F000E20
:102D2C001E6FCDEC08F0B20E02011C6F370E1D6F3A
:102D3C00000E1E6FCDEC08F0BFEC07F00101B76B75
:102D4C00B86BB7C1E9FFB8C1EAFFEE50550A33E1E1
:102D5C00130EB725E96E000EB821EA6EEE50230A69
:102D6C002AE1590E02011C6F3D0E1D6F000E1E6FE5
:102D7C00CDEC08F0350E02011C6F010E1D6FEBEC53
:102D8C0008F0BFEC07F0CBEC0FF0F7EC10F030C113
:102D9C00F7F119EC12F000C060F02AC1F7F119EC50
:102DAC0012F000C061F02BC1F7F119EC12F000C069
:102DBC0068F0B76BB86BB7C1E9FFB8C1EAFFEE506A
:102DCC00440AD8A4BBD0010EB725E96E000EB82179
:102DDC00EA6EEE504D0AD8A4B1D0020EB725E96EBA
:102DEC00000EB821EA6EEE503D0AD8A4A7D0350EDD
:102DFC00F76F010EF86FDAEC10F0800E026E800E99
:102E0C000118025C02E100500608D8A097D0B7C1A7
:102E1C001CF2B8C11DF2EBEC08F0050E0101B72550
:102E2C00E16E000EB821E26EE66A030EB7250201D0
:102E3C001C6F000E0101B82102011D6FCAEC07F0D6
:102E4C0000C01EF101C01FF1000E026E0150025CA9
:102E5C0002E10050010864E2000E01011F5D02E175
:102E6C00150E1E5D5DE21EC13EF01FC13FF000015C
:102E7C006A6B6B6B000E6B5D02E1020E6A5D2EE2FB
:102E8C00030E0101B725006E000EB821016E000182
:102E9C006A510024E96E6B510120EA6EEECFDBF132
:102EAC006B0E6A250101F76F000E00016B21010109
:102EBC00F86FDBC1F9F164EC0FF0020E0B6E040E2F
:102ECC000C6EBA0E0D6E0D2EFED70C2EFCD70B2EE3
:102EDC00FAD7000000016A4B6B2BCCD70101DB6BDE
:102EEC00A10E02011C6F3D0E1D6F000E1E6FCDEC6E
:102EFC0008F0600E0101F76F85EC0FF000C066F072
:102F0C0001C067F00F0E0024E16E000E0120E26E8E
:102F1C00E66A66C01CF267C01DF2EBEC08F009D043
:102F2C000201A90E1C6F3D0E1D6F000E1E6FCDEC25
:102F3C0008F0BFEC07F00101B76BB86BB7C1E9FF44
:102F4C00B8C1EAFFEE50470AD8A428D1010EB72524
:102F5C00E96E000EB821EA6EEE50560AD8A41ED1C6
:102F6C00020EB725E96E000EB821EA6EEE504D0A3E
:102F7C00D8A414D1030EB725E96E000EB821EA6E61
:102F8C00EE503D0AD8A40AD1350EF76F010EF86F3A
:102F9C00DAEC10F0800E0118026E800E025C02E179
:102FAC00080E005CD8A0FAD07C0E02011C6F3C0EFF
:102FBC001D6F000E1E6FCDEC08F0B7C11CF2B8C12E
:102FCC001DF2EBEC08F0060E0101B725E16E000EC8
:102FDC00B821E26EE66A040EB72502011C6F000EE2
:102FEC000101B82102011D6FCAEC07F000C01EF1EF
:102FFC0001C01FF1090E0101B725E16E000EB821C9
:10300C00E26EE66A070EB72502011C6F000E010185
:10301C00B82102011D6FCAEC07F000C020F101C0FD
:10302C0021F1000E026E0150025C02E100500C080E
:10303C00D8B0A6D0000E0101215D02E1180E205D72
:10304C00D8B09ED0000E1F5D02E1050E1E5DD8A00B
:10305C0097D0000E006E1F51005C02E11E510C084F
:10306C00D8A08ED01EC155F01FC156F000016A6B5E
:10307C006B6B000E6B5D02E1020E6A5D2EE2040EBC
:10308C000101B725006E000EB821016E00016A51D6
:10309C000024E96E6B510120EA6EEECFDBF17B0E62
:1030AC006A250101F76F000E00016B210101F86F19
:1030BC00DBC1F9F164EC0FF0020E0B6E040E0C6E1A
:1030CC00BA0E0D6E0D2EFED70C2EFCD70B2EFAD78A
:1030DC00000000016A4B6B2BCCD720C157F021C1EB
:1030EC0058F06A6B6B6B000E6B5D02E1020E6A5D51
:1030FC002EE2070E0101B725006E000EB821016EFD
:10310C0000016A510024E96E6B510120EA6EEECF8A
:10311C00DBF17E0E6A250101F76F000E00016B21B9
:10312C000101F86FDBC1F9F164EC0FF0020E0B6ECC
:10313C00040E0C6EBA0E0D6E0D2EFED70C2EFCD797
:10314C000B2EFAD7000000016A4B6B2BCCD7610E0B
:10315C0002011C6F3C0E1D6F000E1E6FCDEC08F0B3
:10316C007A0E0101F76F85EC0FF000C066F001C01C
:10317C0067F000C01CF201C01DF2EBEC08F009D0A6
:10318C000201990E1C6F3D0E1D6F000E1E6FCDECD3
:10319C0008F0BFEC07F00101B76BB86BB7C1E9FFE2
:1031AC00B8C1EAFFEE504F0AD8A438D2010EB725A9
:1031BC00E96E000EB821EA6EEE50460AD8A42ED263
:1031CC00020EB725E96E000EB821EA6EEE50530AD6
:1031DC00D8A424D2030EB725E96E000EB821EA6EEE
:1031EC00EE503D0AD8A41AD2350EF76F010EF86FC7
:1031FC00DAEC10F0800E0118026E800E025C02E117
:10320C00040E005CD8A00AD2620E02011C6F3A0EAA
:10321C001D6F000E1E6FCDEC08F0940E0101F76FC0
:10322C0085EC0FF000C066F001C067F000C01CF226
:10323C0001C01DF2EBEC08F0BFEC07F00001666B6F
:10324C00676B7F0E0101226FB7C1F7F1B8C1F8F1BE
:10325C00DAEC10F000C01EF101C01FF176D0040EA4
:10326C00B725E96E000EB821EA6E300EEE5C226FC7
:10327C00050EB725E16E000EB821E26EE66A78D035
:10328C00040EB725E96E000EB821EA6EEE502D0A39
:10329C000DE1050EB725E96E000EB821EA6E300E71
:1032AC00EE5C006E00500008226F18D0040EB7259B
:1032BC00E96E000EB821EA6E300EEE5C226F0A0E3B
:1032CC002203F3CF22F1050EB725E96E000EB821CB
:1032DC00EA6E300EEE5C006E00502227060EB7250B
:1032EC00E16E000EB821E26EE66A42D0040EB725FC
:1032FC00E96E000EB821EA6EEE502D0A1BE1050EA8
:10330C00B725E96E000EB821EA6E300EEE5C006E49
:10331C000A0E0002F3CF01F0060EB725E96E000E7F
:10332C00B821EA6E300EEE5C006E015000260050A3
:10333C000008226F070EB725E16E000EB821E26E71
:10334C00E66A16D07F0E226F13D0000E1F1902E111
:10335C00050E1E1984E0000E1F1902E1060E1E193F
:10336C008FE0000E1F1902E1070E1E19BFE0EAD70D
:10337C0022517F0A0AE18D0E02011C6F390E1D6F5E
:10338C00000E1E6FCDEC08F046D14B0E02011C6FE7
:10339C003D0E1D6F000E1E6FCDEC08F022C1F7F133
:1033AC006C0E0101F86F000EF96FF6EC0BF06C0E61
:1033BC0002011C6F000E1D6FEBEC08F0BFEC07F068
:1033CC00B7C1F7F1B8C1F8F1DAEC10F000C01EF19A
:1033DC0001C01FF1EAD0940EF76F000EF86F040EC7
:1033EC00B725E96E000EB821EA6EEECFF9F164EC68
:1033FC000FF0020E0B6E040E0C6EBA0E0D6E0D2E2F
:10340C00FED70C2EFCD70B2EFAD70000950E01011F
:10341C00F76F000EF86FF96B64EC0FF0020E0B6E89
:10342C00040E0C6EBA0E0D6E0D2EFED70C2EFCD7A4
:10343C000B2EFAD70000D0D0940E0101F76F000EBE
:10344C00F86F040EB725E96E000EB821EA6EEECFC8
:10345C00F9F164EC0FF0020E0B6E040E0C6EBA0E4A
:10346C000D6E0D2EFED70C2EFCD70B2EFAD70000AE
:10347C00950E0101F76F000EF86F050EB725E96E7A
:10348C00000EB821EA6EEECFF9F164EC0FF0020EEB
:10349C000B6E040E0C6EBA0E0D6E0D2EFED70C2E8E
:1034AC00FCD70B2EFAD70000960E0101F76F000E19
:1034BC00F86FF96B64EC0FF0020E0B6E040E0C6ED1
:1034CC00BA0E0D6E0D2EFED70C2EFCD70B2EFAD786
:1034DC00000082D0940E0101F76F000EF86F040EFD
:1034EC00B725E96E000EB821EA6EEECFF9F164EC67
:1034FC000FF0020E0B6E040E0C6EBA0E0D6E0D2E2E
:10350C00FED70C2EFCD70B2EFAD70000950E01011E
:10351C00F76F000EF86F050EB725E96E000EB82197
:10352C00EA6EEECFF9F164EC0FF0020E0B6E040EA6
:10353C000C6EBA0E0D6E0D2EFED70C2EFCD70B2E6C
:10354C00FAD70000960E0101F76F000EF86F060E09
:10355C00B725E96E000EB821EA6EEECFF9F164ECF6
:10356C000FF0020E0B6E040E0C6EBA0E0D6E0D2EBD
:10357C00FED70C2EFCD70B2EFAD70000970E0101AC
:10358C00F76F000EF86FF96B64EC0FF0020E0B6E18
:10359C00040E0C6EBA0E0D6E0D2EFED70C2EFCD733
:1035AC000B2EFAD7000018D017D0000E01011F19EE
:1035BC0002E1050E1E19D8B40ED7000E1F1902E138
:1035CC00060E1E19D8B438D7000E1F1902E1070ECB
:1035DC001E19D8B47FD7E8D7CB0E02011C6F3B0E57
:1035EC001D6F000E1E6FCDEC08F0940E0101F76FED
:1035FC0085EC0FF000C066F001C067F000C01CF253
:10360C0001C01DF2EBEC08F0BFEC07F00001666B9B
:10361C00676B22C126F10101B76BB86B9D829E923C
:10362C00000EBA1902E1020EB91909E1970E020156
:10363C001C6F3C0E1D6F000E1E6FCDEC08F0BFEF23
:04364C0014F0FFD7A0
:103DE80010EE1DF0430E006E010E016ED10EF66E40
:0E3DF800380EF76E000EF86E60EC0DF0120043
:10365000204F46465345542063616C696272617421
:10366000696F6E2074656D70657261747572652026
:103670004C4D3335445A2028646F69742065747248
:103680006520636F6D707269732020656E7472655A
:10369000202D3939206574202B3939202920656E79
:0B36A00020656570726F6D203A2000FD
:1036AB0020456570726F6D3A20486F726C6F67655D
:1036BB005F366469676974735F31384632364B32F3
:1036CB00325F5254435F4453333233315F554C4E68
:1036DB005F55444E5F4D656C6F6469655F36306C4A
:1036EB006564735F454550524F4D5F31383039300B
:0936FB00342E696865780D0A009F
:1037040020536F75726365203A20486F726C6F673F
:10371400655F366469676974735F31384632364B66
:1037240032325F5254435F4453333233315F554C2A
:103734004E5F55444E5F4D656C6F6469655F36300E
:103744006C6564735F4344343031355F31383130F4
:0737540031332E630D0A0062
:10375B002047616D652056616C69646174696F6E99
:10376B00204D656C6F646965202047564D3D3038A0
:10377B003B32313C43523E20202864652038483090
:10378B003020E020323148303029206C696D69746B
:10379B006573203520E020313220657420313320D1
:0737AB00E02032330D0A009B
:1037B200204F464653455420636F727265637469A5
:1037C2006F6E2074656D70656172757265204C4D07
:1037D2003335445A2020204F46533D2D33303C434D
:1037E200523E2020286C696D69746573202D393929
:0A37F20020E020393929200D0A00DB
:1037FC002050726F6A6574203A486F726C6F6765FF
:10380C005F366469676974735F31384632364B32A0
:10381C00325F4453333233315F554C4E5F55444E17
:10382C005F4D656C6F6469655F36306C6564732ED3
:08383C006D637070690D0A0054
:1038440020436F6E66696720626974203A205031A4
:10385400384632364B32325F464F53435F696E749B
:1038640065726E655F3878504C4C5F33324D687AC0
:103874002E63666773636820464F53433A33322E90
:0838840030204D487A0D0A00C6
:10388C00204469726563746F7279203A433A5C5FC5
:10389C004D696B726F435C5F4D657350726F6A65F7
:1038AC0074735F4D696B726F435C5F3138463236AF
:1038BC004B32325F486F726C6F67655F36306C6588
:0538CC0064730D0A0009
:1038D1008C3800C73C00FC3700AA3B00443800ABE1
:1038E1003600043700143900EA3A00BD3A00903A34
:0138F10000D6
:0238F2000500CF
:0238F4000000D2
:0138F60000D1
:0938F70030303A30303A30300034
:0939000030302F30302F30300040
:023909000800B4
:02390B001500A5
:01390D000FAA
:04390E0000000000B5
:0139120000B4
:013913003083
:103914002031384632364B32322C20525443204424
:1039240053333233312C36206166666963686575BA
:103934007273203720736567202C756172742020A0
:0D394400313135323030206264730D0A00DD
:103951002046696C746572696E6720414443206D2D
:103961006561737572652062792061726974686D31
:10397100657469632061766572616765206F662091
:0C398100382076616C756573200D0A001B
:10398D002065727265757220736169736965206F48
:10399D00666673657420646F697420657472652042
:1039AD00656E747265203C2D393920657420393966
:0639BD00200D0A2020008D
:1039C300204144435F496E69745F416476616E636D
:1039D30065642028312C303234562920706F75727B
:1039E3002045413134202852433229204C4D333570
:0639F300445A200D0A00F9
:1039F900204475726565204D656C6F646965203A70
:103A090020444D3D31323C43523E202067616D6D6B
:103A190065203220E0203230207365636F6E646563
:053A290073200D0A00EE
:103A2E000D0A2052617070656C20666F726D617444
:103A3E0020646520636465203A2022553B32343B76
:103A4E0030383B31373B30343B31373B3336232232
:043A5E00200D0A002D
:103A6200200D0A4D6F646966204F46465345542027
:103A720063616C6962726174696F6E204C4D33359B
:0E3A8200445A202C2041637475656C3D200071
:103A9000204F6666736574204C4D3335445A20655B
:103AA0006E20656570726F6D20504943203D202D5A
:0D3AB00032372020706F696E74730D0A00AC
:103ABD0020416666696368652054416D622E746F9E
:103ACD0075746573206C657320326D6E2070656E34
:0D3ADD0064616E742031357365630D0A005D
:103AEA00205574696C697365203A2054696E795F50
:103AFA005254435F4453333233315F313830392EB5
:0A3B0A0063206574202E680D0A0088
:103B140020486F72616972652056616C69646174D2
:103B2400696F6E204D656C6F64696520656E2065F4
:093B34006570726F6D203A2000EB
:103B3D002052544320557064617465203A20553BE2
:103B4D0031343B30353B31383B30313B31353B3314
:073B5D0036233C43523E00F9
:103B640020706F757220323420416F7574203230AA
:103B74003137204A657564692031374833360D0A78
:033B84000D0A0027
:103B87000D0A45727265757220737572204A6F75DA
:103B9700722053656D61696E65206A532E204F4B05
:033BA7000D0A0004
:103BAA0020486F726C6F6765203630206C656473CD
:103BBA0020617665632031384632364B32320D0A3F
:013BCA0000FA
:103BCB00204E6F7576656C204F46465345542054F6
:103BDB00656D706572204C4D3335445A203D200085
:103BEB0020706F7572203134204D61692032303175
:103BFB0038204C756E64692031354833360D0A0018
:103C0B000D0A45637269747572652064616E732069
:0F3C1B004453333233312E2E2E204F4B0D0A00DF
:103C2A00204475726565204D656C6F646965206511
:0C3C3A006E20656570726F6D203A2000EE
:103C46002041637469766520736F727469652053C9
:0B3C560051573D31487A3A200D0A001A
:103C6100204E6F7576656C20686F72616972652090
:0B3C71004D656C6F646965203A20000F
:103C7C0047616D652056616C69646174696F6E2073
:0B3C8C004D656C6F646965203A2000F4
:103C97000D0A2042756666657231204F7665726C33
:093CA7006F61642021200D0A0068
:103CB0000D0A2048656C70203A2048656C703C43C2
:073CC000523E20200D0A0016
:103CC700204D696B726F432070726F20372E322E32
:053CD70030200A0D0081
:103CDC00696E697420525443207061722064656669
:053CEC00617574200069
:103CF10020496E6974205254432044533332333186
:053D01003A200D0A004C
:103D06002050726573656E746174696F6E203A2017
:033D16000D0A0093
:103D1900204D656C6F646965203C204D696E2048B3
:023D29003D005B
:103D2B002052652D4C656374757265205254432087
:013D3B000087
:0F3D3C002052415A203630206C6564730D0A0006
:0E3D4B00204E6577204F66667365743D20003C
:0E3D590052544320557064617465203A200076
:0B3D670020496E64657831203D20008B
:0B3D72003F065B4F666D7D077F6F0012
:0A3D7D004D657263726564692E00E3
:093D870056656E64726564690002
:093D900044696D616E6368650011
:083D99002042414420212000DA
:083DA10020204F4B203D2000C3
:083DA9002042414420212000CA
:073DB10053616D65646900B8
:063DB8004C756E64690009
:063DBE004D617264690012
:063DC4004A657564690008
:043DCA0020B04300E2
:043DCE004F46460016
:043DD2004F4E200030
:033DD600202000AA
:033DD9002A480075
:033DDC002A440076
:033DDF002A4D006A
:033DE2002A46006E
:033DE5002A54005D
:020000040030CA
:0D00010038193CFFBF81FF0FC00FE00F401A
:0200000400F00A
:10000000486F726C6F6765203630206C65647320B2
:1000100050494331384632364B323220200A0D00E7
:10002000464F53432033324D485A20202C20202065
:1000300052544320445333323331202C2055415203
:100040005431203131353230302C382C4E2C310D9A
:100050000A00FFFFFFFFFFFFFFFFFFFFFFFFFFFFA4
:10006000447572E9652E4D656C6F3D30330D0A00A5
:1000700056616C69642E4D656C6F3D30383B323192
:100080000D0A0020202000FFFFFFFFFFFFFFFFFF02
:100090004F46533D2D32320000000000000000FFAB
:1000A000FFFFFFFFFFFFFFFFFFFFFFFFFFFFFFFF60
:1000B000FFFFFFFFFFFFFFFFFFFFFFFFFFFFFFFF50
:1000C000FFFFFFFFFFFFFFFFFFFFFFFFFFFFFFFF40
:1000D000FFFFFFFFFFFFFFFFFFFFFFFFFFFFFFFF30
:1003E0007061756C666A756A6F2032303138200032
:1003F000FFFFFFFFFFFFFFFFFFFFFFFFFFFFFFFF0D
:00000001FF
